:1000000025C032C031C030C02FC02EC02DC02CC082
:100010002BC02AC0768D9BA5AEA3A3A3A1A1A1A1AD
:10002000A1A3A3A3A3A3A1A1A1A114C8FF00FDFEA6
:10003000FF031464FFFFFF00FDFEFF00004FFFFD04
:10004000FEFF000000063887FFFDFEFF11241FBEE3
:10005000CFE9CDBF10E0A0E6B0E001C01D92AD3603
:10006000B107E1F7EBD0CAC1CBCF26EB33E003C039
:10007000F9013197F1F70197D8F7089588EE93E0E9
:10008000F4CFCF93C09164008C2F8E5F8F718093DB
:10009000640090916000792F7295707F60E03091DC
:1000A000620020E0622B732B90916100692B90E03D
:1000B00094D16FEF7FEF8C2F90E0CF918EC1CF93D3
:1000C000DF93109264000DC08C2F90E07ED1D82F6A
:1000D0008C2F90E0019679D1DF3F41F4CE5FC09341
:1000E0006400C0916400C03278F30AC0D09361000C
:1000F000982F92959F70909360008170809362001A
:10010000DF91CF910895809161008F5F80936100AE
:1001100090916700891710F0109261000895809106
:10012000610090916700891303C0109261000895E7
:10013000811102C080916C0081508093610008950C
:10014000B49904C081E08093630008951092630025
:10015000089580916200811112C087E0809367004A
:1001600082E490E090936B0080936A0081E390E0DA
:10017000909369008093680080E290E011C084E071
:10018000809367008BE390E090936B0080936A000C
:100190008AE290E0909369008093680089E190E0A2
:1001A0009093660080936500809167008D5F8093D7
:1001B0006C000895A29A81E687B986EC86B9089505
:1001C000811104C0611102C091EA9FBD89BD66BF63
:1001D0000895E0916500F0916600E80FF91FE49141
:1001E000EFBDE0916800F0916900E80FF91F64919C
:1001F000E0916A00F0916B00E80FF91F8491E0CF65
:10020000369A3699FECF85B108951F93CF93DF9329
:10021000C82F14E1D1EA0CC019BC16BF84E690E0E7
:1002200024DFDFBD19BC16BE80E991E01EDFC1509E
:10023000C111F2CFDF91CF911F910895A39A83E668
:1002400087B986EC86B93699FECF369A3699FECFB5
:10025000C5B180E188BBB99AB89A81EA8FBD81E0C7
:1002600083BF6EDF2CDF75DFCB3F48F04CDF809122
:1002700060008F3090F48F5F809360000EC0CF3BA2
:1002800020F04DDF1092600008C010926000809155
:100290006300811102C010926100F3DEBB9AC39A21
:1002A00089DF369AC0E0D0E0EE24E39401EAFF242F
:1002B000FA9480916100E0916A00F0916B00E80F80
:1002C000F11D1491909160009F3079F4D7DE109267
:1002D000600010926100809162008E258093620020
:1002E000D0DE37DF81E091DF42C01E3F89F414E0A9
:1002F000F9BC16BE85E090E0B8DE19BCF6BE81E41C
:1003000090E0B3DE1150A1F780ED92E0AEDE2FC099
:100310001D3FB1F40FBD19BC16BEB0DE71DF70DF3A
:10032000982FE4E1F0E080E02491291708F48F5F32
:10033000319620E0E931F207B9F767DF9FDE17C099
:1003400090E047DFDF3F19F0DF5FDD3350F01F3F04
:1003500041F48091670082508093610090E039DF22
:1003600090DE84EF91E081DE109260008ADE349BA3
:10037000A0CF85B18D3630F5CF5FC83020F1C09168
:10038000610080916700C81798F4CC2311F0C15028
:1003900010C00FBD19BC16BE85B7877E806185BFB2
:1003A00085B7806285BF889585B78F7D85BF01C081
:1003B000C2E08C2F90E00DDFC093610062DE8AEF17
:1003C00090E053DEC0E0369A74CFE199FECF1FBAB9
:1003D0008EBBE09A99278DB3089502D0272F01C0D4
:1003E000262FE199FECF1CBA1FBA8EBB2DBB0FB6CC
:1003F000F894E29AE19A0FBE01960895F894FFCF1F
:00000001FF
